:100000000C9413010C9430010C9430010C943001C9
:100010000C9430010C9430010C9430010C9430019C
:100020000C9430010C9430010C9430010C9430018C
:100030000C9430010C9430010C9430010C9430017C
:100040000C9430010C9430010C9430010C9430016C
:100050000C943001151515151515151515151515D3
:10006000151515151513131313131313121212125A
:1000700012121111111111111111111144454C538A
:10008000455150524755535252454C3F3F3F004215
:100090004C4F434B5320465245452E004552524F3C
:1000A000523A204436340030302C4F4B0032312C41
:1000B00052454144204552524F520032362C57523D
:1000C0004954452050524F54454354204F4E00331D
:1000D000332C53594E544158204552524F520036FA
:1000E000322C46494C45204E4F5420464F554E44E5
:1000F0000036332C46494C4520455849535453004B
:1001000037332C4D4D433249454320444F532056FD
:10011000302E380037342C4452495645204E4F5427
:1001200020524541445900A700AD00BB00CF00DF7D
:1001300000F100000114012C30302C303000455209
:10014000524F523A2053442F4D4D43004552524F87
:10015000523A2046494C452053595354454D004688
:1001600041543136204F4B004641543332204F4BDF
:10017000004552524F523A2046494C4520464F5274
:100180004D415400203C4449523E000000002514DB
:10019000C4170F177F0E0317520B03053D0A750E88
:1001A0004436343F0201032814D7032B144F041F95
:1001B00002221430024D3249D41C31199F1C391BC4
:1001C000FA1AB618AB189E189418543634AA1E6C36
:1001D0001F2814DD1F2B142F1F5A1E22146F1E50B0
:1001E00030302E140000281425142B14520B030554
:1001F00022144F144D32492046494C452045525255
:100200004F52005052470044454C00204D324900A7
:100210002E4D324900002E505247000054415045A7
:1002200020454E442E0011241FBECFE5D8E0DEBF8E
:10023000CDBF10E0A0E6B0E0E2E5F2E402C0059038
:100240000D92AC3BB107D9F715E0ACEBB0E001C0C3
:100250001D92A138B107E1F70E94F31C0C942821EC
:100260000C940000BF92CF92DF92EF92FF920F9317
:100270001F93CF93DF939C0110E000E0EE24FF2456
:10028000C0E6D0E0EEE2BE2E90E2C92E80E3D82E8A
:100290008E2D813021F0843011F0873061F4E12F10
:1002A000FF27002321F0E20FF31FB08203C0E20F0B
:1002B000F31FC0821F5F88819981AA81BB81481783
:1002C00059076A077B0760F4E12FFF27002321F01D
:1002D000E20FF31FD0821EC0E20FF31FC0821AC0CC
:1002E000F901E10FF11DD0820BC080818F5F808307
:1002F00088819981AA81BB81481B590B6A0B7B0BB2
:1003000088819981AA81BB81481759076A077B07B1
:1003100060F701E00894E11CF11C24968AE0E816DD
:10032000F10411F01F5FB4CFDF91CF911F910F91B6
:10033000FF90EF90DF90CF90BF9008951F93CF93E1
:10034000DF93FC01C4E7D0E010E3108307C0808195
:100350008F5F808388819981681B790B9B0144277B
:10036000552788819981AA81BB81281739074A07B7
:100370005B0768F73196249680E0C838D80729F7DC
:10038000DF91CF911F910895CF92DF92EF92FF926C
:100390000F931F93CF93DF93EC0120E030E0D22E38
:1003A0002F5F3F4FFE01ED0DF11D80818032B9F3CB
:1003B000EE24FF2487012AE030E040E050E012C044
:1003C000C801B7010E94DB207B018C018C2D99278D
:1003D000C097AA2797FDA095BA2FE80EF91E0A1F0D
:1003E0001B1FD394FE01ED0DF11DC0808C2D805399
:1003F0008A3030F3C801B701DF91CF911F910F917F
:10040000FF90EF90DF90CF900895009731F0A3E335
:10041000B7E01197F1F70197D1F7089527ED31E093
:10042000482F9927249F812D349F800D911D1124E1
:1004300006971816190614F40197F1F7089580919C
:10044000C004992780FF09C081FF07C09695879552
:100450009695879581709070089581E090E0089559
:100460008091C00481708093C00481E090E0089581
:100470008091C0049927089580E090E008950E943B
:10048000F10460507B4A8240904030F081E08093DC
:10049000C00481E090E008951092C00480E090E0F4
:1004A0000895CF92DF92EF92FF920F931F93382F10
:1004B000D62EC82ECA94862F9927E0E007C0FF27C2
:1004C000EC5AFF4FE4918E0F911DE22F2E2F2F5FDC
:1004D0002317A9F7AA27BB27EE24F82E092F1A2FD6
:1004E0000E94F104E616F70608071907A8F440E091
:1004F000C801B7010E94CE0B0E94520B8093BF042B
:100500000E94520B8093C304C092C204D092BE04D6
:1005100082E08093C10402C01092C0041F910F9129
:10052000FF90EF90DF90CF9008958091C00480FFFE
:100530000EC060E082E10E94510241E06EE870E08E
:1005400080E090E00E94CE0B81E08093C00408958B
:100550000F931F93CF93DF93AC018091C004282F9A
:10056000332720FF36C023FF34C024FD32C0EA0108
:100570008A01025E1F4F0E94520B89938091C10431
:100580008F5F8093C104C017D107A9F7882389F42E
:100590008091BF04882329F06091C3040E94510216
:1005A00005C08091C00480618093C00481E090E028
:1005B00012C00E94520B182F0E94520B982F80914C
:1005C000C1048E5F8093C104112381F79F3F49F3DB
:1005D000EDCF80E090E0DF91CF911F910F910895D2
:1005E0008091C00480FD03C080E090E0089561E048
:1005F00082E10E94510289E08093C00481E090E092
:100600000895EF92FF920F931F93CF93DF93CDB78F
:10061000DEB7EE970FB6F894DEBF0FBECDBF7C01FC
:100620008091C00480FD0DC08E01015E1F4F4AE025
:1006300050E06CE970E0C8010E948720A8016AE0E0
:10064000A0C00E94950282E18F8F82E288A392E08F
:100650009EAF0E94520B9EAD803A09F480E2923127
:1006600009F494C08E01015E1F4FF801E90FF11DDE
:1006700080839F5F993160F3A80169E180E090E099
:10068000F701099543E050E060E270E0C8010E9484
:10069000902082E28AA30E94F00258C08A818823B7
:1006A00009F454C08E010D5D1F4F4AE150E060E235
:1006B00070E0C8010E94902094E0FE013496D801B9
:1006C0008081803A29F08D939F5F31969431C1F7F4
:1006D000FE01E90FF11D82E2878F898187708630E4
:1006E00008F085E063E0869FB001112464587F4FD5
:1006F00043E050E0CE01C5960E948720998196FF85
:1007000002C08CE388AF97FD02C08AE289AF2D8DCD
:100710008E8D9927982F8827820F911D23E0883E80
:10072000920710F023E00AC08436910510F022E011
:1007300005C020E08A30910508F021E0AE01415E5D
:100740005F4F420F511D6BE1F7010995CE010196F4
:100750000E94A802882309F0A1CF8E01015E1F4FDD
:100760004CE050E06FE870E0C8010E9487204DE047
:1007700050E060E270E0CE018B960E949020A801CC
:1007800069E180E090E0F701099504C082E289AB5D
:1007900093E15ECFEE960FB6F894DEBF0FBECDBFED
:1007A000DF91CF911F910F91FF90EF900895CF921D
:1007B000DF92EF92FF920F931F93CF93DF93CDB70A
:1007C000DEB76E970FB6F894DEBF0FBECDBF6C01DB
:1007D00060E170E00E94C620082F0E94F0024CC029
:1007E000898187708150823008F046C011E020E096
:1007F00030E0402F5527B70114C0A82FBB27F601C2
:10080000EA0FFB1F90819F3351F09A3299F010E06C
:10081000A60FB71FFD018381981709F411E02F5F20
:100820003F4F822F2417350719F0112331F711C0DC
:10083000112379F0801759F4003148F410E0FE01DB
:10084000E00FF11D8481803A21F411E00DC01123E5
:1008500059F47E010894E11CF11CC7010E94A80212
:10086000882309F0BDCF0AC06B818A810E945102A2
:1008700083E08093C00402C010E0EBCF812F992762
:100880006E960FB6F894DEBF0FBECDBFDF91CF914D
:100890001F910F91FF90EF90DF90CF9008951F93DD
:1008A0000E941F02882311F080E01AC00E94520BA0
:1008B000182F8091C1048F3F79F48091BF04882361
:1008C00029F06091C3040E94510209C08091C004C4
:1008D00084608093C00403C08F5F8093C104812F24
:1008E00099271F9108958093BC00807711F0D998C3
:1008F0000895D99A08956115710581059105B1F49E
:100900008091BC0082FF09C02091F7043091F80467
:100910004091F9045091FA0423C02091FF043091D2
:10092000000540910105509102051AC062507040C7
:10093000804090402091C8043091C9044427552735
:100940000E94DB209B01AC018091F7049091F80498
:10095000A091F904B091FA04280F391F4A1F5B1FB8
:10096000CA01B90108952091F7043091F80440912B
:10097000F9045091FA04621B730B840B950B2091C0
:10098000C8043091C904442755270E9406212E5FD0
:100990003F4F4F4F5F4FCA01B9010895EF92FF9249
:1009A0000F931F939B01AC018091BC00E090FB046E
:1009B000F090FC040091FD041091FE0482FF04C03D
:1009C000220F331F441F551F9927852F742F632F24
:1009D0006E0D7F1D801F911F1F910F91FF90EF9053
:1009E00008958091BC0083FD05C060E070E080E068
:1009F00090E008956091EB047091EC048091ED0417
:100A00009091EE0408958091BC0083FD03C081E0C5
:100A100090E0089560E070E02091F3043091F404D8
:100A20004091F5045091F6048091EB049091EC0410
:100A3000A091ED04B091EE04281739074A075B072F
:100A400010F061E070E0CB01089580E00E94730433
:100A50008FEF9FEFAFEFBFEF8093C4049093C50477
:100A6000A093C604B093C7048093B0009093B100E4
:100A7000A093B200B093B3008093B4009093B500FC
:100A8000A093B600B093B70008958091BC00992759
:100A9000089560910305709104058091050590917A
:100AA000060508958091C8049091C9040895609145
:100AB000CA047091CB048091CC049091CD04089528
:100AC00060910B0570910C0580910D0590910E05BC
:100AD00008956091C4047091C5048091C6049091FA
:100AE000C70408950F931F93CF93DF93CDB7DEB75D
:100AF0002C970FB6F894DEBF0FBECDBF8C014CE033
:100B000050E0BC01CE0101960E94B72049814E32CF
:100B1000B9F48A818E3211F492E008C091E006C0E7
:100B2000F801E90FF11D80E280839F5F9B30C0F3E5
:100B300045C04D9101964E3239F4232F3F5F1AC0C4
:100B400080E090E0DE011296282F442359F0F8014E
:100B5000E80FF91F4083382F3F5F8730910549F731
:100B6000232F08C0382F06C0F801E20FF11D80E2E4
:100B700080832F5F2830C0F3FE01E30FF11D8181D8
:100B80008E3271F43F5F0CC0FE01E30FF11D8181D5
:100B9000882379F0F801E20FF11D80833F5F2F5F1A
:100BA0002B3090F306C0F801E20FF11D80E2808344
:100BB0002F5F2B30C0F3C8010E94D120F8011386AB
:100BC0002C960FB6F894DEBF0FBECDBFDF91CF914C
:100BD0001F910F910895D998D19A84E190E00E94D5
:100BE0000502D99A08950E942E1D99270895809193
:100BF000BC0086FF15C04091AC005091AD006091E3
:100C0000B4007091B5008091B6009091B7000E9439
:100C1000F305882329F08091BC008F7B0E94730428
:100C20000895EF92FF920F931F93CF93DF937B0171
:100C30008C010E94F705E091AC00F091AD0080E0DE
:100C400092E011920197E9F7C801B7010E947B0475
:100C50006093B4007093B5008093B6009093B70092
:100C6000C0E0D0E012C04091AC005091AD00609166
:100C7000B4007091B5008091B6009091B7006E0FEE
:100C8000711D811D911D0E94F305EC2F21962E2FC1
:100C900033278091C8049091C9042817390718F3A5
:100CA000DF91CF911F910F91FF90EF900895EF92F8
:100CB000FF920F931F937B018C018091B400909160
:100CC000B500A091B600B091B7008E159F05A007A2
:100CD000B10751F00E94F705E092B400F092B50020
:100CE0000093B6001093B7001F910F91FF90EF9003
:100CF0000895DF92EF92FF920F931F938091BC00B3
:100D000085FF35C0E090B000F090B1000091B200D6
:100D10001091B3004091AE005091AF00C801B701EF
:100D20000E94F305882319F121E0D22E17C080918B
:100D3000030590910405A0910505B0910605E80E04
:100D4000F91E0A1F1B1F4091AE005091AF00C80151
:100D5000B7010E94F305882351F0D3948091CE040B
:100D6000D81628F38091BC008F7D0E9473041F91D8
:100D70000F91FF90EF90DF9008950E94811D9927B9
:100D80000895AF92BF92CF92DF92EF92FF920F93AE
:100D90001F93CF93DF937B018C014091AC00509166
:100DA000AD000E94BD068091AC009091AD00EC01B9
:100DB0002B9645E050E068E870E0C6960E94A920B6
:100DC000892B19F080E090E09AC08091BC0081608E
:100DD0000E947304AB80BC80CC24DD24AE0CBF1C0D
:100DE000C01ED11E6D81862F9927EB84FC848E9DB9
:100DF00090018F9D300D9E9D300D11244427552765
:100E00002A0D3B1D4C1D5D1D2093FF0430930005F2
:100E100040930105509302058E819F8174E0969561
:100E200087957A95E1F7AA27BB27280F391F4A1F14
:100E30005B1F2093F7043093F8044093F904509318
:100E4000FA0400271127E0920305F09204050093AD
:100E50000505109306058A81482F55275093C9042C
:100E60004093C804A092FB04B092FC04C092FD041D
:100E7000D092FE046093CE0428853985C901AA2743
:100E8000BB278093CA049093CB04A093CC04B09367
:100E9000CD04232B61F48D899E89AF89B88D809311
:100EA000CA049093CB04A093CC04B093CD04CA01A0
:100EB0009C01442755276091CA047091CB0480910E
:100EC000CC049091CD040E9406212093CA04309353
:100ED000CB044093CC045093CD0410920B05109298
:100EE0000C0510920D0510920E051092C40410927C
:100EF000C5041092C6041092C70481E090E0DF910F
:100F0000CF911F910F91FF90EF90DF90CF90BF9006
:100F1000AF9008954F925F926F927F929F92AF929F
:100F2000BF92CF92DF92EF92FF920F931F93CF93D6
:100F3000DF932B013C014091AC005091AD000E9429
:100F4000BD068091AC009091AD00EC012B9645E080
:100F500050E06EE870E08E5A9F4F0E94A920892BC6
:100F600019F080E090E074C08091BC0085600E9420
:100F70007304EB80FC8000271127E40CF51C061D90
:100F8000171D9D80692D772788279927A98CBA8CF2
:100F9000CB8CDC8CA60195010E94DB206E0D7F1DA1
:100FA000801F911F6093F7047093F8048093F904F5
:100FB0009093FA04A0920305B0920405C09205052F
:100FC000D09206052A8133273093C9042093C804A0
:100FD000E092FB04F092FC040093FD041093FE04E5
:100FE0009092CE04442755276D897E898F89988DEC
:100FF0000E9406212093CA043093CB044093CC0472
:101000005093CD048DA19EA1AA27BB27840D951DC9
:10101000A61DB71D8093070590930805A0930905A9
:10102000B0930A0589A19AA1ABA1BCA180930B053D
:1010300090930C05A0930D05B0930E058093C40406
:101040009093C504A093C604B093C70481E090E0D8
:10105000DF91CF911F910F91FF90EF90DF90CF9094
:10106000BF90AF909F907F906F905F904F9008954A
:101070000E94EB0580E00E9473048FEF9FEFAFEFBB
:10108000BFEF8093B0009093B100A093B200B093F3
:10109000B3008093B4009093B500A093B600B093D2
:1010A000B7004091AC005091AD0060E070E080E08E
:1010B00090E00E94BD06E091AC00F091AD00E250DE
:1010C000FE4F8081EE5FF140853509F042C0E1506E
:1010D000FE4F8081EF5FF1408A3AD9F5E254FE4F2E
:1010E00080818068803811F584818D3038F48B30B0
:1010F00088F4843029F08630C9F402C08E30B1F40F
:101100008091BC0082608093BC006085718582857F
:1011100093851BC08091BC0082608093BC00608579
:101120007185828593850E948A0711C060E070E016
:1011300080E090E00E948A07882319F081E090E027
:10114000089560E070E080E090E00E94C106992779
:10115000089580E090E00895EF92FF920F931F931F
:101160007B018C018091B4009091B500A091B600F4
:10117000B091B7008E159F05A007B10791F00E94AE
:10118000F705E092B400F092B5000093B60010931A
:10119000B7004091AC005091AD00C801B7010E946A
:1011A000BD061F910F91FF90EF900895FA016083A3
:1011B000718382839383158214820E947B040E9430
:1011C000AC088091AC009091AD000895EF92FF9231
:1011D0000F931F937B018C018091B0009091B1001F
:1011E000A091B200B091B3008E159F05A007B10782
:1011F00091F00E9479064091AE005091AF00C80175
:10120000B7010E94BD06E092B000F092B1000093D9
:10121000B2001093B3001F910F91FF90EF900895CB
:10122000AF92BF92CF92DF92EF92FF920F931F93F4
:101230007B018C0159016A010E94CE040E94E608DC
:101240008091BC002091AE003091AF0082FF22C09F
:10125000F701EF77F070EE0FFF1FEE0FFF1FE20FA9
:10126000F31F80819181A281B38180709070A07002
:10127000B07F2FEF3FEF4FEF5FE0A222B322C422F7
:10128000D5228A299B29AC29BD2980839183A283F9
:10129000B38308C0F701F070EE0FFF1FE20FF31FDA
:1012A000B182A0828091BC0080620E9473041F9171
:1012B0000F91FF90EF90DF90CF90BF90AF90089587
:1012C000AF92BF92CF92DF92EF92FF920F931F9354
:1012D0009B01AC018091BC0082FF20C0220F331F14
:1012E000441F551F1BC09B014427552797E0EE0C58
:1012F000FF1C001F111F9A95D1F72E0D3F1D401F97
:10130000511F6AC09B0144275527B02FAF2D9E2D3A
:101310008827280F391F4A1F5B1F5EC0A32EB42EDB
:10132000C52EDD24860175016091FB047091FC04DB
:101330008091FD049091FE046E0D7F1D801F911F12
:101340000E94E6088091BC002091AE003091AF0071
:1013500082FF14C0F90160E070E080819181A28178
:10136000B381BF700097A105B10509F4BCCF6F5FD1
:101370007F4F34966038710581F0EFCFF90160E05E
:1013800070E080819181892B09F4BCCF6F5F7F4F22
:10139000329681E060307807A1F70894E11CF11CD7
:1013A000011D111D8091030590910405A091050573
:1013B000B0910605E816F9060A071B0718F0EE2497
:1013C000FF248701EA14FB040C051D0509F0ACCFCE
:1013D00020E030E040E050E0CA01B9011F910F91D8
:1013E000FF90EF90DF90CF90BF90AF900895EF9275
:1013F000FF920F931F937B018C010E94CE040E94E9
:10140000E6088091BC002091AE003091AF0082FFD1
:1014100017C0F701EF77F070EE0FFF1FEE0FFF1F01
:10142000E20FF31F60817181828193819F70683F19
:101430002FEF72072FEF82072FE09207C8F014C03A
:10144000F701F070EE0FFF1FE20FF31F8081918113
:101450009C01B90188279927683F3FEF730730E067
:10146000830730E0930720F060E070E080E090E0D8
:101470001F910F91FF90EF9008955F926F927F926E
:101480008F929F92AF92BF92CF92DF92EF92FF9294
:101490000F931F93CF93DF93582E8091BC0083FF4F
:1014A000EFC08091F3049091F404A091F504B09101
:1014B000F604EC01D1709C01AD012F5F3F4F4F4FFF
:1014C0005F4F2093F3043093F4044093F50450935A
:1014D000F604213031054105510509F49BC02097E0
:1014E00009F098C08091EB049091EC04A091ED0478
:1014F000B091EE04E090EF04F090F0040091F1045C
:101500001091F204281739074A075B0760F5C801F4
:10151000B7010E94B3045B016C010894E11CF11C4B
:10152000011D111DC801B7010E94B304A616B7061C
:10153000C806D90649F4E092EF04F092F004009353
:10154000F1041093F20466C0C601B5010E94F709C8
:101550000E947B046093EF047093F0048093F10485
:101560009093F20457C0370148010894611C711C24
:10157000811C911CC401B3010E94B3045B016C0186
:10158000C801B7010E94B3046A157B058C059D054F
:1015900049F46092EF047092F0048092F10490920A
:1015A000F2042EC0C601B5010E9460097B018C01C6
:1015B000611571058105910509F462C06091EF0420
:1015C0007091F0048091F1049091F2040E94B304B0
:1015D000A80197010E9410092FEF3FEF4FEF5FEF37
:1015E000C801B7010E941009C801B7010E947B041D
:1015F0006093EF047093F0048093F1049093F204ED
:101600006091EF047091F0048091F1049091F204E4
:101610000E9457066091EF047091F0048091F104EC
:101620009091F2040E94AC088091AC009091AD00C2
:10163000C80FD91F58828091BC0080650E94730436
:101640002091F3043091F4044091F5045091F60494
:101650008091EB049091EC04A091ED04B091EE0424
:1016600082179307A407B50740F42093EB04309347
:10167000EC044093ED045093EE0481E090E002C04E
:1016800080E090E0DF91CF911F910F91FF90EF905C
:10169000DF90CF90BF90AF909F908F907F906F9092
:1016A0005F900895AF92BF92CF92DF92EF92FF9238
:1016B0000F931F93CF93DF930E940305882319F0A4
:1016C00080E090E060C08091F3049091F404A091D8
:1016D000F504B091F604EC01D1700196A11DB11D85
:1016E0008093F3049093F404A093F504B093F6046C
:1016F0000197A105B105A9F1209799F5E090EF04B4
:10170000F090F0040091F1041091F204C801B701C7
:101710000E94B3045B016C010894E11CF11C011DE3
:10172000111DC801B7010E94B304A616B706C8066A
:10173000D90649F4E092EF04F092F0040093F1042A
:101740001093F2040EC0C601B5010E94F7090E9471
:101750007B046093EF047093F0048093F104909302
:10176000F2046091EF047091F0048091F104909183
:10177000F2040E94AC088091AC009091AD00C80FBB
:10178000D91F88819927DF91CF911F910F91FF90E9
:10179000EF90DF90CF90BF90AF9008954F925F92FF
:1017A0006F927F928F929F92AF92BF92CF92DF9271
:1017B000EF92FF920F931F93CF93DF93CDB7DEB7D6
:1017C00024970FB6F894DEBF0FBECDBF6B017C012E
:1017D0008091BC0083FFADC04130D9F0413080F032
:1017E000423009F0A6C08091EB049091EC04A091E6
:1017F000ED04B091EE048C199D09AE09BF0915C026
:10180000C092F304D092F404E092F504F092F6044E
:1018100014C08091F3049091F404A091F504B09168
:10182000F6048C0D9D1DAE1DBF1D8093F304909397
:10183000F404A093F504B093F6042091E3043091EE
:10184000E4044091E9045091EA048090F3049090FC
:10185000F404A090F504B090F60481149104A1045E
:10186000B10471F0D501C4019170A070B0700097FF
:10187000A105B10529F4089481089108A108B108CF
:10188000C901AA27BB273C0155244424CA01AA2721
:10189000BB27480E591E6A1E7B1E0091C80410917A
:1018A000C9049801322F2227330F44275527C50139
:1018B000B4010E94062169017A01B9E0B694A794A7
:1018C00097948794BA95D1F789829A82AB82BC8229
:1018D0004801AA24BB240BC0C301B2010E94F7092E
:1018E0002B013C010894C108D108E108F108C1149A
:1018F000D104E104F10481F7C301B2010E947B0429
:101900007B018C0169817A818B819C81A501940185
:101910000E940621E60EF71E081F191FE092EF0431
:10192000F092F0040093F1041093F20481E090E04F
:1019300002C080E090E024960FB6F894DEBF0FBEA0
:10194000CDBFDF91CF911F910F91FF90EF90DF906E
:10195000CF90BF90AF909F908F907F906F905F904F
:101960004F900895CF93DF93EC018D818F5F8D832E
:10197000803108F442C01D822C812F5F2C8380911E
:10198000BC0082FD22C088819981AA81BB81009719
:10199000A105B105D1F48091FF0490910005A091BB
:1019A0000105B0910205820F911DA11DB11D20916D
:1019B000F7043091F8044091F9045091FA04821729
:1019C0009307A407B507C8F034C033278091C80433
:1019D0009091C9042817390780F01C8268817981A9
:1019E0008A819B810E94F709688379838A839B831C
:1019F0006115710581059105E1F0688179818A8120
:101A00009B810E947B042C81620F711D811D911DA1
:101A10000E94AC088D81682F772735E0660F771F0D
:101A20003A95E1F78091AC009091AD00680F791F75
:101A300002C060E070E0CB01DF91CF910895CF93B9
:101A4000DF93CDB7DEB726970FB6F894DEBF0FBE93
:101A5000CDBFAE014F5F5F4F0E94D6080EC08081A0
:101A60008E3239F0882361F0853E19F080E090E0F5
:101A700009C0CE0101960E94B20CFC01892B79F7B6
:101A800081E090E026960FB6F894DEBF0FBECDBF82
:101A9000DF91CF910895EF92FF920F931F93CF9311
:101AA000DF93CDB7DEB763970FB6F894DEBF0FBEF6
:101AB000CDBF7C018E01095F1F4F4CE050E0C80193
:101AC0000E94B7201B8AC8010E9472056091C4045D
:101AD0007091C5048091C6049091C704AE014F5F18
:101AE0005F4F0E94D60823C0F8018081882319F433
:101AF00000E010E01FC0853EB1F0F80183858F3013
:101B000091F04BE050E0BE01695F7F4FC8010E9439
:101B1000A920892B41F4D701F80180E201900D92B0
:101B2000815041F0FBCFCE0101960E94B20C8C0196
:101B3000892BD1F6C80163960FB6F894DEBF0FBEAD
:101B4000CDBFDF91CF911F910F91FF90EF9008953E
:101B50000F931F93CF93DF93CDB7DEB7A7970FB641
:101B6000F894DEBF0FBECDBF8091BC00992783FFE4
:101B7000ABC084FFA9C06FEC74E0CE0108960E9450
:101B80004B0D8C01892B39F40E9479060E94F705D0
:101B900080E090E09FC08091EB049091EC04A091D4
:101BA000ED04B091EE04F801848F958FA68FB78F66
:101BB000CE0101960E9456124E815527A5E0440F92
:101BC000551FAA95E1F78D819927982F8827990F9E
:101BD000990F990F2F812695820F911D480F591F3C
:101BE0002A813327E5E0220F331FEA95E1F78B8145
:101BF0009C818C5B9740982F8827990F6981860F6D
:101C0000911D280F391FF801468B452F5527478B0B
:101C1000208F832F9927818F228B838B8091BC000B
:101C200080640E9473048091BC0082FF48C0609170
:101C30000705709108058091090590910A050E9499
:101C4000AC08E091AC00F091AD00E851FE4F8FEF91
:101C50008083E091AC00F091AD00E751FE4F8083AE
:101C6000E091AC00F091AD00E651FE4F8083E09131
:101C7000AC00F091AD00E551FE4F8083E091AC00E7
:101C8000F091AD00E451FE4F8083E091AC00F09103
:101C9000AD00E351FE4F8083E091AC00F091AD00C8
:101CA000E251FE4F8083E091AC00F091AD00E15134
:101CB000FE4F80838091BC0080640E9473048091F9
:101CC000BC008F7E0E9473040E9479060E94F70573
:101CD00081E090E0A7960FB6F894DEBF0FBECDBFAF
:101CE000DF91CF911F910F9108950E94A80D8091CF
:101CF000BC00877F0E94730481E090E008950F93F9
:101D00001F938C010E94A80DB8018FEC94E00E94F3
:101D10004B0D892B19F480E090E035C00091BC0098
:101D20002091E9043091EA0402FF12C06091E304BB
:101D30007091E40488279927CB01772766274427E9
:101D40005527620F731F841F951F0E947B0405C0D7
:101D5000B901882799270E947B041092F3041092FE
:101D6000F4041092F5041092F6046093EF0470935B
:101D7000F0048093F1049093F204802F88600E9415
:101D8000730481E090E01F910F9108956F927F920C
:101D90008F929F92AF92BF92CF92DF92EF92FF927B
:101DA0000F931F93CF93DF93CDB7DEB7A0970FB6F6
:101DB000F894DEBF0FBECDBFBC01CE0101960E94DC
:101DC0004B0D8C01009709F445C06090B4007090F1
:101DD000B5008090B6009090B700FC018489958989
:101DE000AA27BB276C01BB24AA24828D938DAA2726
:101DF000BB27A80EB91ECA1EDB1E8385803131F4B5
:101E0000C601B5010E941F0D882321F1C401B30151
:101E10000E94AC0885EEF80180838091BC0080644C
:101E20000E947304C601B5010E94F7097B018C0171
:101E300020E030E040E050E0C601B5010E9410090A
:101E400057016801E114F1040105110559F781E01A
:101E500090E002C080E090E0A0960FB6F894DEBF5C
:101E60000FBECDBFDF91CF911F910F91FF90EF90EB
:101E7000DF90CF90BF90AF909F908F907F906F90AA
:101E80000895CF92DF92EF92FF920F931F93CF931B
:101E9000DF93CDB7DEB7AD970FB6F894DEBF0FBEB8
:101EA000CDBF7C018B013EE0C32ED12CCC0EDD1EBC
:101EB000C6010E944B0D892B19F5B701C6010E947E
:101EC0004B0D7C01892BE1F04CE050E0B8018E0114
:101ED0000F5F1F4FC8010E94B7201D86C8010E94D6
:101EE0007205F701D8018BE00D9001928150E1F766
:101EF0008091BC0080640E94730481E090E002C085
:101F000080E090E0AD960FB6F894DEBF0FBECDBF77
:101F1000DF91CF911F910F91FF90EF90DF90CF90C5
:101F20000895CF93DF93CDB7DEB7A0970FB6F8949F
:101F3000DEBF0FBECDBFFC0180818F3249F480919E
:101F40000B0590910C05A0910D05B0910E052FC0C9
:101F5000BF01CE0101960E944B0D892B89F18C8522
:101F600084FF2EC08B8D9C8D9C01442755278D8925
:101F70009E89AA27BB27DC0199278827280F391FAC
:101F80004A1F5B1F2093C4043093C5044093C604CA
:101F90005093C7048091BC0082FF15C02115310504
:101FA0004105510581F482E090E0A0E0B0E080932B
:101FB000C4049093C504A093C604B093C70403C09F
:101FC00080E090E002C081E090E0A0960FB6F89427
:101FD000DEBF0FBECDBFDF91CF910895CF92DF92CC
:101FE000EF92FF920F931F93CF93DF93CDB7DEB79E
:101FF00026970FB6F894DEBF0FBECDBF7B018C01D4
:10200000AE014F5F5F4F0E94D6080EC0F60180817F
:10201000853EE9F18823D9F1E980FA800B811C81A2
:10202000CE0101960E94B20C6C01892B79F7809148
:10203000BC0082FD05C0E114F1040105110539F170
:10204000C801B7010E9460099B01AC0161157105CF
:1020500081059105E1F069837A838B839C83C801B4
:10206000B7010E94100969817A818B819C812FEFD1
:102070003FEF4FEF5FEF0E94100969817A818B81FA
:102080009C810E941106C090AC00D090AD00C601AA
:1020900026960FB6F894DEBF0FBECDBFDF91CF916D
:1020A0001F910F91FF90EF90DF90CF9008956F9266
:1020B0007F928F929F92AF92BF92CF92DF92EF92D8
:1020C000FF920F931F93CF93DF93CDB7DEB7E497C3
:1020D0000FB6F894DEBF0FBECDBF4C01BC01CE01E0
:1020E00045960E944B0D892B09F095C06091C40460
:1020F0007091C5048091C6049091C7040E94EE0FB0
:102100007C01892B09F487C06091C4047091C504D7
:102110008091C6049091C7040E9460095B016C0124
:10212000611571058105910509F475C08E01085F7F
:102130001F4F4CE050E0B401C8010E94B7201C8A38
:10214000C8010E947205CE0101960E9456128E812E
:10215000682E772455E0660C771C5A95E1F78D813F
:102160009927982F8827990F990F990F2F812695D6
:10217000820F911D680E791E8A81682F772735E0BE
:10218000660F771F3A95E1F78B819C818C5B9740B6
:10219000982F8827990F2981820F911D680F791F29
:1021A000A70198018BE0D9010D909D01FA010192E0
:1021B000AF018150C1F780E2F7018387148615864D
:1021C0006686472D55274787608B272F3327218B1E
:1021D000628B238BC601AA27BB27958B848B668ACB
:1021E000478B608F218FB38EA28E148E158E168E24
:1021F000178E8091BC0080640E9473042FEF3FEF24
:102200004FEF5FEFC601B5010E941009C4010E94A3
:102210007F0E992702C080E090E0E4960FB6F89414
:10222000DEBF0FBECDBFDF91CF911F910F91FF9009
:10223000EF90DF90CF90BF90AF909F908F907F9066
:102240006F9008954F925F926F927F928F929F92BC
:10225000AF92BF92CF92DF92EF92FF920F931F93B4
:10226000CF93DF93CDB7DEB7E4970FB6F894DEBF18
:102270000FBECDBF4C01BC01CE0145960E944B0D57
:10228000892B09F0FAC06091C4047091C504809153
:10229000C6049091C7040E94EE0F7C01892B09F4BB
:1022A000ECC06091C4047091C5048091C604909103
:1022B000C7040E9460095B016C016115710581050D
:1022C000910509F4DAC08E01085F1F4F4CE050E021
:1022D000B401C8010E94B7201C8AC8010E9472057F
:1022E000CE0101960E9456128E81682E772455E009
:1022F000660C771C5A95E1F78D819927982F8827CE
:10230000990F990F990F2F812695820F911D680EB5
:10231000791E8A81682F772735E0660F771F3A95F7
:10232000E1F78B819C818C5B9740982F8827990FD0
:102330002981820F911D680F791FA70198018BE0F9
:10234000D9010D909D01FA010192AF018150C1F7B1
:1023500080E1F701838714861586162D6686472D42
:102360005527842E4787962E608B272F3327022FE1
:10237000218B628B238BC601AA27BB272C01958B4F
:10238000848B668A478B608F218F3501B38EA28E36
:10239000148E158E168E178E8091BC0080640E945C
:1023A0007304C601B5010E941106E091AC00F091E2
:1023B000AD00AF0124E930E08BE0D9010D909D0123
:1023C000DA010D92AD018150C1F780E18387148657
:1023D000158616878786908A018B928A038B558A89
:1023E000448A168B878A908E018F738E628E148E2C
:1023F000158E168E178EB096AF0120EA30E08BE076
:10240000D9010D909D01DA010D92AD018150C1F706
:1024100080E183871486158616878786908A018BCC
:10242000928A038B8091C4049091C504A091C60444
:10243000B091C704CD01AA27BB27958B848B168B3F
:10244000878A908E018F8091C4049091C504938FE8
:10245000828F148E158E168E178E8091BC0080642C
:102460000E9473042FEF3FEF4FEF5FEFC601B501FE
:102470000E94100981E090E002C080E090E0E496C4
:102480000FB6F894DEBF0FBECDBFDF91CF911F9185
:102490000F91FF90EF90DF90CF90BF90AF909F9003
:1024A0008F907F906F905F904F900895FC0181E036
:1024B0008083818387ED97E09383828381E18483A6
:1024C0008EE185831682089588B3887F88BB87B3A1
:1024D000887F87BB10920F0588E0809310050895D0
:1024E000B998BA9884E60E940E0281E090E00895BF
:1024F0000F931F93CF93DF93082F162FC0E0D0E0E8
:1025000086B38023112329F090E0882309F491E019
:10251000892F882319F080E090E011C082E00E94AA
:102520000E0221968DEFC83ED80751F7BA98B99898
:1025300084E080930F05B09BFECF81E090E0DF91B7
:10254000CF911F910F910895B99A86E40E940E02CF
:10255000BA9886E40E940E0261E084E00E9478123C
:1025600090E0811191E081E09827892F99270895C3
:1025700060E084E00E947812882319F080E090E007
:102580000895B99886E40E940E02BA9A86E40E94E1
:102590000E0281E090E008950F931F93082F162FED
:1025A00061E082E00E947812882309F03FC0BA9867
:1025B00060E082E00E9478128823C1F5112379F04F
:1025C00088EC0E940E0261E082E00E94781288236B
:1025D00069F560E082E00E947812882339F584E191
:1025E0000E940E0210E0BA9A00FF02C0B99801C022
:1025F000B99A86E40E940E02BA9886E40E940E02FE
:102600001F5F183011F00695EECFBA9AB99884E1A1
:102610000E940E0261E082E00E94781290E0811137
:1026200091E081E09827892F992702C080E090E00F
:102630001F910F91089561E00E94CC12882319F434
:1026400080E090E008950E94A41220E030E088230A
:1026500011F021E030E0C901089560E00E94CC1241
:1026600099270895FF920F931F93CF93DF931092B2
:102670000F0560E084E00E947812882309F044C0CE
:10268000B998C0E0D0E003C08AE00E940E02B29B7D
:1026900005C02196C531D105B9F702C0C43180F01B
:1026A00080910F05816080930F05B99A86E40E949E
:1026B0000E02B99861E084E00E947812882321F527
:1026C000B09905C080910F05826080930F0510E0DE
:1026D00000E060E084E00E9478128823A9F4B19BB6
:1026E00003C080E8F82E01C0FF2461E084E00E946E
:1026F0007812882349F416951F290F5F083049F78F
:10270000B99A812F992702C080E090E0DF91CF91A4
:102710001F910F91FF9008950E94321399270895F9
:10272000CF92DF92FF920F931F93CF93DF936C01B1
:10273000B0996FC0B99ABA9882E30E940E020E94C3
:102740003213982F80910F0582FD72C08091100581
:102750008062981769F50E943213982F80910F05B7
:1027600082FD66C0F6019083892F807F803619F440
:10277000FF2412E055C09F3309F450C000E010E080
:10278000E601F02E0E943213982F80910F0582FDF2
:102790004FC080910F0581FF02C09F33E9F10F5FA9
:1027A0001F4F21960932110509F442C09883E9CFE1
:1027B000809110058064981721F50E943213982F9C
:1027C00080910F0582FD34C0F6019083FF2411C073
:1027D000B29B0FC00E943213982F80910F0582FD8B
:1027E00027C0F7E2FF1520F1F601EF0DF11D9183EF
:1027F000F394B09BEDCF0E94B8128823C9F013E088
:102800000FC084E60E940E02B998BA98B09906C02B
:10281000FDCFB998BA9802C011E002C0FF2410E0C1
:1028200084E60E940E02F601F1A6812F992702C0CC
:1028300084E090E0DF91CF911F910F91FF90DF90A6
:10284000CF90089581E090E0089581E090E00895B0
:1028500082E090E0089580E090E008951F930E9448
:10286000520B8334C1F40E94520B8633A1F40E94B0
:10287000520B843381F410E00E94520B1F5F17311A
:10288000D9F70E94030520E030E0882311F421E00D
:1028900030E0C90102C080E090E01F9108951092DD
:1028A00011050E94750E81E090E0089510921305C5
:1028B0008FEF8093110586E0809312050E94D01D52
:1028C000882321F00E9425050E9438080E944505B2
:1028D00080FF06C08091BD00882311F01092110581
:1028E00008950E945614D898D09A84E190E00E94EE
:1028F0000502D89A8A98929AD298DA9AD398DB9A53
:102900000895CF93DF93EC010E948C13FE0109958B
:1029100080910F0580FD04C080910F0582FFF4CFE8
:10292000DF91CF910895FF920F931F93CF93DF9381
:102930008C01F62EEA0180913C0590913D050596AB
:10294000860F911D90933D0580933C0580913C0539
:1029500090913D050E942D1380913C0590913D057D
:10296000892F99270E942D13802F0E942D13012F4C
:10297000110F110B802F0E942D1300E007C0FE01E4
:10298000E00FF11D80810E942D130F5F0F15B9F725
:1029900080E00E942D13DF91CF911F910F91FF9046
:1029A0000895EF92FF921F93CF93DF93EC017B0189
:1029B00005C0812F0E942D13882339F0FE0109954F
:1029C000182FF70109958823A1F3812F0E941B136B
:1029D000DF91CF911F91FF90EF9008950F931F9378
:1029E0008C0181E098E090933D0580933C0581E067
:1029F0000E942D1388E00E942D1383E994E1F801D1
:102A0000099580E00E942D1380E00E941B131F9106
:102A10000F910895CF93DF93E0911205FF27EE0FFA
:102A2000FF1FE95DFE4FC591D49102C00E942D1396
:102A3000FE01219684918823C9F7C7E3D1E0FE0106
:102A400084910E942D132196F1E0CC33DF07B9F772
:102A5000FE0184910E941B13DF91CF9108950F9383
:102A60001F93CF93DF9380913F05803419F411E0D9
:102A700001E002C010E000E0CFE3D5E06AE370E0DF
:102A8000CE010E949720009719F0182F1C1B1F5F82
:102A90001123C1F0912F20916705412F55270DC0BB
:102AA000E92FFF27DF01A41BB50BA25CBA4FE25C44
:102AB000FA4F8181FD0181839F5F291788F7211BD0
:102AC00020936705802F9927DF91CF911F910F9158
:102AD0000895FF920F931F93CF93DF93EC01109211
:102AE000130580913F058F3549F4809140058F355E
:102AF00029F48FEF8093110581E095C08091BD008E
:102B0000882321F00E94450580FD07C087E080935F
:102B100012058FEF8093110588C080913F058432A4
:102B200009F46AC08F3591F480911105882341F42E
:102B300088EB90E00E94910F882309F476C05CC076
:102B40008F3F09F472C01092110556C00E942F15D4
:102B5000882311F085E067C080911105882309F072
:102B600051C020E030E0909167054EE70AC0E82FA1
:102B7000FF27E25CFA4F81818F3F09F441832F5F89
:102B80003F4F822F291798F38FE395E00E94910F12
:102B9000882391F58FE395E00E947F0E882309F446
:102BA0003DC080916705C82FDD27C45CDA4F00EA7D
:102BB00011E041E0F42E43E050E0B801CE010E9464
:102BC0007A20892B39F0F3940B5E1F4F85E0F816BD
:102BD00091F728C0F8013396259134918FE395E061
:102BE000F9010995882351F0F0921105F801359605
:102BF00085919491892BB1F083E015C01092110555
:102C000084E011C08F3F89F0FE01399625913491FF
:102C10008FE395E0F9010995882321F484E08093FE
:102C2000120503C082E0809313056FE375E084E131
:102C300095E00E94A220DF91CF911F910F91FF900C
:102C40000895CF93DF9388E080931005CA9905C05B
:102C500080911005816080931005CB9905C080910B
:102C60001005826080931005829B08C0D89AD99A7B
:102C70008FEF809311051092BD000CC08091BD00B4
:102C8000882341F482E390E00E940502D8980E94D4
:102C90005614D89A8EE395E00E949013282F843022
:102CA00009F4AEC0882309F4ABC0D898E0911105AF
:102CB000EF3F19F4C0E0D0E006C085E1E89FE001F5
:102CC0001124C557DE4FE0916705FF27E25CFA4FFC
:102CD000118280913E05382F3F709927807F907038
:102CE000803E910509F483C0803F910529F080362C
:102CF000910509F084C017C03F3079F4209749F05E
:102D0000FE013796259134918FE395E0F9010995FD
:102D100001C087E08093120572C010921205CE01A7
:102D20000E9469156CC0233009F033C03F3029F48C
:102D30000E940A151092120562C08091130581301D
:102D400029F40E94561486E797E104C0843029F4E0
:102D50008AE497E10E94EE1452C0882311F0209774
:102D600019F40E9470124BC0823059F4FE013F9654
:102D700065917491FE013D96859194910E94D114C4
:102D80003EC0833009F03BC0FE0135968591949199
:102D9000E1CF223009F033C0209729F482E294E198
:102DA0000E948114B6CF80911305853031F0809157
:102DB0001205843011F085E013C0FE013B96259189
:102DC000349184E195E0F9010995882311F482E0BA
:102DD00007C010921205FE0171968591949104C06E
:102DE0008093120582E294E10E94811408C020972A
:102DF00031F0FE01739685919491FC010995D89A62
:102E0000DF91CF9108950F931F938C010E94C60EFE
:102E1000C8010E94571099271F910F9108951F9381
:102E2000CF93DF9310913F056AE370E08FE395E065
:102E30000E949720009731F1EC012196133521F47F
:102E4000CE010E94C60E0FC0123581F46DE370E012
:102E5000CE010E949720FC01892BA1F01192BE01A6
:102E6000CF010E94410F882379F00CC01E3411F06D
:102E700083E00BC0CE010E941F1C882331F482E046
:102E80008093110580E001C084E09927DF91CF9104
:102E90001F910895EF92FF920F931F93CF93DF93AB
:102EA000CDB7DEB763970FB6F894DEBF0FBECDBFC8
:102EB0007C0142E150E061E771E08E010F5F1F4F3E
:102EC000C8010E948720A80162E180E090E0F7013C
:102ED000099563960FB6F894DEBF0FBECDBFDF91A4
:102EE000CF911F910F91FF90EF9008950F931F9333
:102EF000CF93DF93CDB7DEB763970FB6F894DEBFFD
:102F00000FBECDBF8C010E944505982F8091BD005A
:102F1000882351F44DE050E06EE371E0CE0101965C
:102F20000E9487206DE01EC0292F332720FD0AC094
:102F300042E150E06CE471E0CE0101960E948720EE
:102F400062E110C0CE01019622FF05C048E050E0CA
:102F500068E671E004C048E050E06FE571E00E946F
:102F6000872068E0AE014F5F5F4F80E090E0F8019E
:102F7000099563960FB6F894DEBF0FBECDBFDF9103
:102F8000CF911F910F910895EF92FF920F931F938E
:102F9000CF93DF93CDB7DEB76E970FB6F894DEBF51
:102FA0000FBECDBF7C0143E050E060E270E0CE0197
:102FB00007960E94902082E28A870E946905AE01EE
:102FC0004F5F5F4F0E94D6088AC08081882309F432
:102FD0008AC0853E09F47FC083858F3009F47BC0A9
:102FE000883019F4AF016BE027C084FF28C09E0130
:102FF000255F3F4FAF0188E0DA010D90AD01D901A7
:103000000D929D018150C1F780E28B8BDE015496B9
:10301000389683E001900D928150E1F782E28F8B28
:1030200046E050E064E871E0CE0148960E948720B7
:10303000AE01495F5F4F67E180E090E04AC0848D58
:10304000958DA68DB78D81509C4FAF4FBF4F5AE0E5
:10305000B695A795979587955A95D1F79C01B7E2B4
:1030600020313B0718F02FE037E204C083E0283E10
:10307000380710F060E00BC02436310510F061E035
:1030800006C02A30310510F062E001C063E0AE01F5
:10309000455F5F4F8F0188E0D8010D908D01DA0107
:1030A0000D92AD018150C1F78EE28B8BDE015496FB
:1030B000389683E001900D928150E1F782E28F8B88
:1030C000AE01495F5F4F461B51094D5F5F4F625F25
:1030D000C901F7010995CE0101960E94B20CFC01CD
:1030E000892B09F072CF8091BD00882381F48E0175
:1030F000095F1F4F4DE050E06EE371E0C8010E9490
:103100008720A8016DE080E090E0F70109956E96B8
:103110000FB6F894DEBF0FBECDBFDF91CF911F91E8
:103120000F91FF90EF900895809168058E7F8093B6
:1031300068050E94750E81E090E00895982F8091B7
:10314000680580FD03C080E090E00895892F0E940B
:103150003D0A992708958091680580FD03C081E0AC
:1031600090E008950E9403059927089580916805CD
:1031700080FD03C080E090E008950E94520B9927E3
:103180000895CF92DF92EF92FF920F931F93CF9308
:10319000DF937C016B010E940305882371F50E9477
:1031A000520B082F0E94520B8A3339F5E70110E0C9
:1031B0000E94520BE114F10409F088831F5F2196ED
:1031C0001C30B1F70E94520B8A33B9F4E60110E0CB
:1031D0000E94520BC114D10409F088831F5F21960D
:1031E0001031B1F70E94520B8D3039F40E94520B0E
:1031F0008A3019F4802F992702C080E090E0DF9197
:10320000CF911F910F91FF90EF90DF90CF90089595
:10321000EF92FF921F93CF93DF93EC017C0110E0BC
:103220000E94520BE114F10409F088831F5F21967C
:103230001031B1F70E94520B8D3019F080E090E010
:103240000AC00E94520B90E08A3009F091E081E0C0
:103250009827892F9927DF91CF911F91FF90EF90A9
:103260000895CF92DF92EF92FF920F931F93CF9327
:10327000DF93CDB7DEB76B970FB6F894DEBF0FBE06
:10328000CDBF6C011092680589E695E00E947F0E23
:10329000882361F44EE050E064EF71E08E010F5F2F
:1032A0001F4FC8010E948720A80120C082E18983A6
:1032B00002E20A83CE0103960E940819182F0B8B95
:1032C00044E050E06BE072E0CE0144960E9487201B
:1032D0007E010894E11CF11C112371F44EE050E0D2
:1032E00064EF71E0C7010E948720A7016EE080E0D3
:1032F00090E0F601099531C0A70167E180E090E018
:10330000F601099580E289838A830B830C8B8D8B70
:103310001EC0BE016C5F7F4F80E090E00E94C1182C
:10332000803519F463E072E004C0843481F467E00E
:1033300072E043E050E0CE0146960E948720AE0145
:103340004F5F5F4F68E180E090E0F60109950E94D1
:1033500003058823F1F20E94750E6B960FB6F89460
:10336000DEBF0FBECDBFDF91CF911F910F91FF90B8
:10337000EF90DF90CF900895AF92BF92CF92DF92FF
:10338000EF92FF920F931F93CF93DF93CDB7DEB7EA
:103390002D970FB6F894DEBF0FBECDBF6C01109213
:1033A000680548E050E0BC018E010F5F1F4FC80167
:1033B0000E94B72068E070E0C8010E94C6208830F3
:1033C00058F4992748E050E0481B590B60E270E040
:1033D000800F911F0E94902045E050E066E172E06E
:1033E000CE0109960E948720EE24FF2411C0089484
:1033F000E11CF11C85E6E816F10409F465C0812F93
:103400006AE00E94FA20191B105D1F83905D988767
:103410001E2D5E010894A11CB11CC5010E947F0EE7
:10342000882329F789E695E00E947F0E882309F416
:103430004BC080E090E00E940819882309F444C042
:1034400042E060E070E080E090E00E94CE0B80E51A
:103450000E943D0A8AE30E943D0A8501F80181919C
:103460008F010E943D0ACE010D9608171907B1F78A
:103470008AE30E943D0AF601F0808601EE24FF20D7
:1034800031F08F2D0E943D0AF801F18003C080E2E7
:103490000E943D0AE3940F5F1F4FF0E1EF1679F7AA
:1034A0008DE00E943D0A8AE00E943D0A0E94750E4E
:1034B000CE0101960E94571080916805816080932B
:1034C000680581E090E002C080E090E02D960FB6A4
:1034D000F894DEBF0FBECDBFDF91CF911F910F914A
:1034E000FF90EF90DF90CF90BF90AF900895BF9284
:1034F000CF92DF92EF92FF920F931F93CF93DF93C0
:103500006C017B01EA01B22E222339F089E695E0B5
:103510000E947F0E882341F45EC040E060E070E0CE
:1035200080E090E00E94CE0B80E090E00E940819BD
:10353000882309F450C060E170E0CE010E94C620EB
:10354000082F01C00150002309F448C0FE01E00F1C
:10355000F11D319780818032A9F340C0B701C601C7
:103560000E94C1188035D1F5F7013F9620E104C0D3
:1035700021503197222319F080818032C9F390E0E5
:1035800011E012C0A92FBB27FE01EA0FFB1FE0814B
:10359000EF3349F0EA32C1F010E0AE0DBF1D8C915F
:1035A000E81709F411E09F5F901719F0112351F704
:1035B00007C0112329F010E0021711F411E004C034
:1035C0000E940305882351F2BB2011F00E94750E62
:1035D000812F992705C080E090E002C010E0F0CF75
:1035E000DF91CF911F910F91FF90EF90DF90CF90DF
:1035F000BF900895EF92FF920F931F93CF93DF93A5
:10360000CDB7DEB76C970FB6F894DEBF0FBECDBF57
:103610007C011092680521E0AC01BE01635F7F4F21
:103620008E010F5F1F4FC8010E94771A882361F037
:10363000C8010E94C60EC8010E94571080916805FB
:1036400081608093680503C0C7010E94BC19809106
:1036500068059927817090706C960FB6F894DEBF5C
:103660000FBECDBFDF91CF911F910F91FF90EF90D3
:1036700008950F931F93CF93DF93CDB7DEB76C9769
:103680000FB6F894DEBF0FBECDBF1092680521E0E3
:10369000AC01BE01635F7F4F8E010F5F1F4FC801FA
:1036A0000E94771A882351F0C8010E947F0E882358
:1036B00029F0809168058160809368058091680594
:1036C0009927817090706C960FB6F894DEBF0FBE8C
:1036D000CDBFDF91CF911F910F910895CF92DF92CF
:1036E000EF92FF920F931F93CF93DF93CDB7DEB787
:1036F00060970FB6F894DEBF0FBECDBF8C016B0193
:10370000809168058E7F8093680589E695E00E9428
:103710007F0E882319F480E090E02EC020E0A801FD
:10372000BE016F5F7F4F80E090E00E94771A882390
:1037300011F410E01DC041E06EEE7FEF8FEF9FEFC0
:103740000E94CE0BF601F0808601EE24FF2031F0BE
:103750008F2D0E943D0AF801F18003C080E20E9493
:103760003D0AE3940F5F1F4FF0E1EF1679F711E088
:103770000E94750E812F992760960FB6F894DEBFD0
:103780000FBECDBFDF91CF911F910F91FF90EF90B2
:10379000DF90CF900895DF92EF92FF920F931F93E7
:1037A000CF93DF93CDB7DEB76C970FB6F894DEBF3B
:1037B0000FBECDBF7C01809168058E7F8093680528
:1037C00089E695E00E947F0E882319F480E090E05E
:1037D00028C0DD2420E0A701BE01635F7F4F8E017A
:1037E0000F5F1F4FC8010E94771A8823B1F041E094
:1037F0006FED7FEF8FEF9FEF0E94CE0B8DE20E9467
:103800003D0A0E94750EC8010E94C60E89E695E029
:103810000E947F0E81E0D82EDDCF0E94750E8D2D87
:1038200099276C960FB6F894DEBF0FBECDBFDF911F
:10383000CF911F910F91FF90EF90DF900895CF925D
:10384000DF92FF920F931F93CF93DF93CDB7DEB735
:103850002D970FB6F894DEBF0FBECDBF6C018091DF
:1038600068058E7F8093680548E050E0B6018E01C0
:103870000F5F1F4FC8010E94B72068E070E0C801C9
:103880000E94C620883058F4992748E050E0481B31
:10389000590B60E270E0800F911F0E94902045E07C
:1038A00050E060E172E0CE0109960E948720C801D5
:1038B0000E947F0E882329F00E94750E85E090E01B
:1038C00030C0C8010E945710882319F482E090E0AC
:1038D00028C0F601F0808601DD24FF2031F08F2D15
:1038E0000E943D0AF801F18003C080E20E943D0A77
:1038F000D3940F5F1F4FF0E1DF1679F78DE00E9440
:103900003D0A8AE00E943D0A0E94750EA9E6B5E0D4
:10391000FE0131968DE001900D928150E1F780E03B
:1039200090E02D960FB6F894DEBF0FBECDBFDF91AD
:10393000CF911F910F91FF90DF90CF9008951F932B
:10394000CF93DF93FC0110816AE370E00E9497201F
:10395000009711F1EC012196133521F4CE010E945C
:10396000CB1B0FC0123581F46DE370E0CE010E94D5
:103970009720FC01892B81F01192BE01CF010E949A
:103980006E1B882359F008C01E3411F083E007C075
:10399000CE010E941F1C03C080E001C084E0992773
:1039A000DF91CF911F9108951F93FC01019000209A
:1039B000E9F73197E81BF90B3D9718F080E090E0AC
:1039C00010C0BC0189E695E00E94A2201092680513
:1039D00080E090E00E940819182F0E94750E812F38
:1039E00099271F9108950E94641278940E94311EB5
:1039F0000E94D01D0E9438080E9471140E94211656
:103A0000FDCFCF93DF93CFEFDFEF01C021978FEF93
:103A10000E94411E882311F42097C1F7CE01CD2BBF
:103A200011F081E090E0DF91CF9108951F93CF9343
:103A3000DF93182FCFEFDFE001C021978FEF0E94B7
:103A4000411E811711F02097C1F7CE01CD2B11F047
:103A500081E090E0DF91CF911F910895EF92FF9266
:103A60000F931F93CF93DF937B018C01EA0186991B
:103A70001AC0C49888E50E94411E89E0EE0CFF1C24
:103A8000001F111F8A95D1F7C801B7010E94471E78
:103A90008FEF0E94411E80E00E94161D882331F4A2
:103AA000C49A1092BD0080E090E024C08EEF0E9486
:103AB000411E00E010E089910E94411E0F5F1F4FE0
:103AC00082E000301807B9F78FEF0E94411E8FEF98
:103AD0000E94411E8FEF0E94411E8F70853001F7BA
:103AE0000E94011D8823E1F2C49A8FEF0E94411EBB
:103AF0008FEF90E0DF91CF911F910F91FF90EF90AA
:103B00000895CF92DF92EF92FF920F931F93CF937E
:103B1000DF937B018C016A01C49881E50E94411EFC
:103B200099E0EE0CFF1C001F111F9A95D1F7C801F8
:103B3000B7010E94471E8FEF0E94411E80E00E9445
:103B4000161D882329F08EEF0E94161D882331F45C
:103B5000C49A1092BD0080E090E019C0C0E0D0E0AF
:103B60008FEF0E94411EF60181936F012196F2E0D2
:103B7000C030DF07A9F78FEF0E94411E8FEF0E9430
:103B8000411EC49A8FEF0E94411E8FEF90E0DF919B
:103B9000CF911F910F91FF90EF90DF90CF900895FC
:103BA0001F938E98969A1092BD00C49A10E08FEFE2
:103BB0000E94411E1F5F1A30D1F7C49880E40E9412
:103BC000411E60E070E080E090E00E94471E85E9C1
:103BD0000E94411E81E00E94161D882399F1C49A1B
:103BE0008FEF0E94411EC4981FEF81E40E94411E86
:103BF00060E070E080E090E00E94471E8FEF0E943E
:103C0000411E115080E00E94161D882319F41123D3
:103C1000C9F0EBCF1123B1F0C49A8FEF0E94411E7F
:103C2000C49880E50E94411E60E072E080E090E070
:103C30000E94471E8FEF0E94411E80E00E94161DC9
:103C4000882321F4C49A80E090E009C0C49A8FEFE1
:103C50000E94411E8FEF8093BD008FEF90E01F9177
:103C60000895C79AC49ABF9ABE98BD9ABC9A6C9A96
:103C7000689869986B986A986D986E9A8EB18FB1B2
:103C800008958FB9779BFECF8FB1992708959B0137
:103C9000AC015FB9779BFECF8FB14FB9779BFECF59
:103CA0008FB13FB9779BFECF8FB12FB9779BFECFF6
:103CB0008FB1089580917E05992780FF09C081FF0B
:103CC00007C0969587959695879581709070089511
:103CD00081E090E0089580917E0599270895809174
:103CE0007E05817080937E0581E090E0089580914B
:103CF0007E0580FD03C080E090E0089540E060E430
:103D000070E080E090E00E94CE0B89E080937E0519
:103D1000109277051092760580917805909179053B
:103D2000892B19F081E090E0089589E180937E0568
:103D300081E090E0089580917E0580FF0AC040E018
:103D400068E270E080E090E00E94CE0B81E080931A
:103D50007E0508950F931F9310927E050E94F10433
:103D60006034710581059105E8F140E060E070E0A4
:103D700080E090E00E94CE0B0E94520B833491F5BC
:103D80000E94520B863371F50E94520B843351F519
:103D900040E062E270E080E090E00E94CE0B0E9482
:103DA000520B9927909379058093780540E063E260
:103DB00070E080E090E00E94CE0B009178051091B9
:103DC00079050E94520B9927982F8827082B192BC9
:103DD000109379050093780581E080937E0581E05A
:103DE00090E002C080E090E01F910F9108950F9342
:103DF0001F93CF93DF93AC0180917E05282F33274B
:103E000020FF26C023FF24C024FD22C0EA018A012E
:103E1000005E1F4F0E94520B8993C017D107D1F744
:103E20008091760590917705019690937705809320
:103E3000760520917805309179058217930729F44A
:103E400080917E05806180937E0581E090E002C0D4
:103E500080E090E0DF91CF911F910F9108950E9433
:103E60005A1E882311F020E034C080917A05909189
:103E70007B052FEF8E3F920749F420917F058FEF4E
:103E80009FEF90937B0580937A0523C08F5F9F4FB0
:103E900039F42091800510927B0510927A0519C0A3
:103EA0000E94520B482F80917A0590917B050196D4
:103EB00090937B0580937A0520917C0530917D0558
:103EC0008217930729F480917E05846080937E0594
:103ED000242F822F99270895EF92FF920F931F931B
:103EE000CF93DF93CDB7DEB7E6970FB6F894DEBF7A
:103EF0000FBECDBF7C010E949B1E82E1898382E2BE
:103F00008A838E010D5F1F4F0E94520B803A09F485
:103F100080E2F80181938F01CE014696E817F907F8
:103F200099F712E21B8BAE014F5F5F4F66E180E0B5
:103F300090E0F701099580E289838A831B831C8BBB
:103F40000E94771E17C08F898823A1F0888D88234F
:103F500089F0DE011496FE01B79680E101900D9282
:103F60008150E1F7AE014F5F5F4F64E180E090E088
:103F7000F7010995CE0147960E94F71E882319F78D
:103F800049E050E06CE172E08E010F5F1F4FC80105
:103F90000E948720A80169E080E090E0F701099580
:103FA000E6960FB6F894DEBF0FBECDBFDF91CF917E
:103FB0001F910F91FF90EF900895CF92DF92EF92B3
:103FC000FF920F931F93CF93DF93CDB7DEB7A097E8
:103FD0000FB6F894DEBF0FBECDBF8C01FC0101907F
:103FE0000020E9F73197FE2EF81A80E18F1510F4C2
:103FF00090E1F92E0E94771E6AC08981882309F416
:1040000066C08A81882309F462C081E0E82E20E03E
:10401000A60114C0A22FBB27F801EA0FFB1F3081B5
:104020003F3359F03A3241F1EE24A40FB51FFD01A0
:104030008089381711F4B1E0EB2E2F5F2F1519F09E
:10404000EE2041F70FC0EE2069F0FFE0FF15A0F071
:10405000EE24FE01EF0DF11D8189803219F4A1E0FB
:10406000EA2E0AC06E010894C11CD11CC6010E9430
:10407000F71E882311F62DC06B8160937F054C815C
:10408000409380058EEF9FEF90937B0580937A0598
:104090002D8133278E819927982F8827282B392B1C
:1040A00077275527542F4427642B752B261B370B56
:1040B00030937D0520937C0569857A858B859C8569
:1040C00040E00E94CE0B83E080937E0502C0EE2488
:1040D000C9CF8E2D9927A0960FB6F894DEBF0FBEDC
:1040E000CDBFDF91CF911F910F91FF90EF90DF90A7
:1040F000CF900895FB01DC0104C08D9105908019DB
:1041000021F441505040C8F7881B990B0895FB01DA
:10411000DC0102C005900D9241505040D8F708953F
:10412000DC0101C06D9341505040E0F70895FC015F
:104130008191861721F08823D9F79927089531971F
:10414000CF010895FB01DC0101900D920020E1F701
:104150000895FB01DC014150504030F08D910190F9
:10416000801919F40020B9F7881B990B0895FB01F9
:10417000DC014150504048F001900D920020C9F7F9
:1041800001C01D9241505040E0F70895FC0161507C
:10419000704001900110D8F7809590958E0F9F1F69
:1041A0000895DC016C9161566A3108F0605E6F5BC6
:1041B0006D93C1F70895629FD001739FF001829FB4
:1041C000E00DF11D649FE00DF11D929FF00D839FA6
:1041D000F00D749FF00D659FF00D9927729FB00D43
:1041E000E11DF91F639FB00DE11DF91FBD01CF0156
:1041F00011240895991B79E004C0991F961708F0BF
:10420000961B881F7A95C9F780950895A1E21A2E0A
:10421000AA1BBB1BFD010DC0AA1FBB1FEE1FFF1F6A
:10422000A217B307E407F50720F0A21BB30BE40BBA
:10423000F50B661F771F881F991F1A9469F7609501
:104240007095809590959B01AC01BD01CF010895BB
:02425000FFCF9E
:1042520000CA9A3B00E1F5058096980040420F00A3
:10426200A086010010270000E8030000640000009F
:104272000A00000001000000464154313600464168
:10428200543332002E202020202020202020200005
:104292002E2E20202020202020202000BE00BE0222
:0C42A200FFFFFFFFFFFFFFFF2E2E0000BC
:00000001FF
